:10000000B4011E2AB416B41EB412B4190B28B415C8
:100010004620031832280830A3005B20A20DA30B52
:100020000D28B41E3D2065206120B41A32203720EF
:1000300022080310192AB416B41EB4123419252844
:10004000FE39B50034150310192A341A2D28A600DC
:10005000341646200318322826084E20031832286A
:10006000B41E192A3D20652034113412B411380809
:100070008400360884178004432838088400360931
:1000800080058417800544284528192A37206520D3
:100090001D223D2061203508B4190138A200083026
:1000A000A300A20D03183720031C3D20652061200A
:1000B000A30B512837206520380884003608000536
:1000C000FF3E390884003709402839088400370882
:1000D0003A28A400B5172730A30010307B20033046
:1000E000A300E8307B20A30164307B20A3010A3009
:1000F0007B2024088628A2002508A1002408A0004F
:10010000E2212008031DB513B51B0800303EA700EF
:100110000711871007108316071187100710F0309A
:10012000860583122708B418B3283A30A100983006
:10013000C1213330A600C8201330A1008830C1216E
:10014000C8206430C021C8206430C0212230A600FD
:10015000C8202830B2200C30B2200630B220B414AF
:100160002708B3283414A600341CC1288710033C88
:10017000031CC628C6200730A100D030C1210314BB
:1001800008003414FE3C0319192A8714A60E341CE7
:1001900034100715F030860526080F39860407113C
:1001A000A60E3418C8283230C02103140800640099
:1001B000ED200318D7286021A8010830A300612191
:1001C000ED200318A80AAB1EA801A20CA30BDF2880
:1001D000AB1AA213612122080800380884003608EF
:1001E00084178004841300052B1B3606FF3E08008D
:1001F000A401A501B5121422D33E0319B5162D3E54
:10020000C63E0318FB280A3E031CFB28A20003106D
:10021000240DA000250DA100200DA10DA407031899
:10022000A10A2108A507A40DA50D2208A4070318FB
:10023000A50AA903031923291422C63E031823295A
:100240000A3E03180629B51E2A29A409A509A40AED
:100250000319A50A2408192A0408A60038088400EE
:10026000F030B5050830A70003100318B50A462181
:10027000A60CA70B35290000AB1A350C46211C2211
:10028000031446212F08A3002E08B4298413AB1FA2
:100290005529000836042B1F3606800084170008F5
:1002A0003604031C36068000612900083604031C4E
:1002B00036062B1B36068000841736098005612917
:1002C00035172B081F39003EA1002A080E3E0318DF
:1002D000A10A351FC1293513A0000230DD21C12933
:1002E000B51329080319B5170530A8002730A30056
:1002F000103086210330A300E8308621A30164304A
:100300008621A3010A30862124088D29A200250810
:10031000A1002408A000E2212008A000A8030319DE
:10032000B513290803199729280203180800200883
:10033000031DB513B51B0800303E142AA000A00D04
:10034000A00DA00D3830A005813020049F000030A2
:10035000A1003230C1211F151F19AC291E08A100B0
:1003600083161E08192AA301A200FF30A207031C4E
:10037000A307031C192A0330A100E630C121B529C7
:10038000A101FC3EA000A109031CCC29FF30000004
:10039000A0070318C729A0076400A10FC6290800F9
:1003A000013EA7000A30A200A301E221A70BD52934
:1003B000240808000310A10CA00CFF3E0318DA2942
:1003C0002008192A1030A600A501A401210DA40DB2
:1003D000A50D2208A4022308031C230FA50203185D
:1003E000F8292208A40723080318230FA5070310E0
:1003F000A00DA10DA60BE6292008192A1030A8008F
:10040000A101A001A70CA60C031C0C2A2208A0071E
:1004100023080318230FA107A10CA00CA50CA40C02
:10042000A80B022A2408192A840031088A003008FF
:100430008200831303138312640008008316DF30E5
:10044000850084309F0070308600811387018312FD
:100450008A11F02BFE308A01872001308A01872023
:1004600050308A01872061308A0187206C308A01F0
:1004700087206D308A01872020308A0187204C3008
:100480008A01872069308A0187206E308A0187209F
:100490006B308A01872020308A01872031308A0121
:1004A00087202E308A01872033308A01872001304F
:1004B000A300F4308A01B421FE308A018720C030C5
:1004C0008A01872050308A01872072308A01872074
:1004D0006F308A01872064308A01872075308A0155
:1004E000872063308A01872065308A018720643045
:1004F0008A01872020308A01872062308A01872084
:1005000079308A01872020308A01872069308A016A
:1005100087207A308A01872075308A018720403011
:100520008A0187200130A300F4308A01B421080039
:1005300000308A019E21C2002108C3000A308A01CE
:10054000B32101308A019E21C6002108C7000A306C
:100550008A01B32108004008A6004108A700043022
:10056000A200A3018A01FE21BA002508BB000730C2
:10057000B8001030B6000730B9000830B700A0301E
:100580008A011D203B088A011D203A088A011D208E
:1005900043088A011D2042088A011D2047088A015C
:1005A0001D2046088A011B200A308A01B321080059
:1005B0004008A6004108A7000430A200A3018A0158
:1005C000FE21BA002508BB000730B8001030B60085
:1005D0000730B9000830B700A0308A011D203B0861
:1005E0008A011D203A088A011D208A010420C300C7
:1005F0008A010420C2008A010420C7008A01022067
:10060000C6000A308A01B32108000730B800403024
:10061000B6005430AA00AB01AE01AF016F308A01C1
:100620002D210D308A012D210A308A012D2108004B
:100630004208A0004308A10003308A01D021CB006A
:100640004208A0004308A10002308A01D021CC005A
:100650004208A0004308A10001308A01D021CD004A
:100660004208A0004308A10000308A01D021C40044
:10067000C5014608A0004708A10003308A01D02127
:10068000CE004608A0004708A10002308A01D02110
:10069000CF004608A0004708A10001308A01D02100
:1006A000D0004608A0004708A10000308A01D021F0
:1006B000C800C9010730B8004030B6005430AA0065
:1006C000AB01AE01AF0153308A012D212C308A01DC
:1006D0002D21A9014B08A400A5012C30B000013048
:1006E000B1008A017021A9014C08A400A5012C3099
:1006F000B0000130B1008A017021A9014D08A400A9
:10070000A5012C30B0000130B1008A017021A9018F
:100710004408A4004508A5002C30B0000130B10009
:100720008A0170212C308A012D21A9014E08A400D4
:10073000A5012C30B0000130B1008A017021A9015F
:100740004F08A400A5012C30B0000130B1008A018F
:100750007021A9015008A400A5012C30B00001307F
:10076000B1008A017021A9014808A4004908A50028
:100770002C30B0000130B1008A0170210D308A01A7
:100780002D210A308A012D2108000730B800803061
:10079000B6005430AA00AB018A01D720733C8A11FD
:1007A000031DCC2B08000730B8008030B600543051
:1007B000AA00AB018A01D720CA0008000730B800A0
:1007C0008030B6005430AA00AB010530A900D73004
:1007D000B000B1018A01F820BE002508BF00080062
:1007E0008501860187018A012A228A01C5233230C8
:1007F0008A01B3218A0105238A01D323FE308A01AD
:10080000872001308A0187204A088A0187203230F8
:100810008A01B3218A0105238A01DE23FE308A0181
:100820008720C0308A0187203F08A5003E088A0142
:10083000692032308A01B3218A0118238A01F52BFD
:0608400063008A01202C78
:02400E00753DFE
:024214000000A8
:00000001FF
